:100000000C9457000C9474000C9474000C947400BD
:100010000C9474000C9474000C9474000C94740090
:100020000C9474000C9474000C9474000C94740080
:100030000C9474000C9474000C9474000C94CF0213
:100040000C9474000C9474000C9474000C94740060
:100050000C9474000C9474000C9474000C94740050
:100060000C9474000C9474000C9474000C944B0366
:100070000C9425030C9474000C9474000101090085
:100080000001010100000100040506070302010050
:100090000102030000000000010101010000000056
:1000A0001020408008040201020408011B041124EE
:1000B0001FBECFEFCDBFDFE3DEBF28E3A0E0B8E394
:1000C00001C01D92A33CB207E1F710E0C7E5D0E004
:1000D00004C02197FE010E946704C635D107C9F705
:1000E0000E9479030C9487040C940000AF92BF9295
:1000F000CF92DF92EF92FF920F931F93CF93DF93F4
:100100006C017B018B01040F151FEB015E01AE1822
:10011000BF08C017D10759F06991D601ED91FC9144
:100120000190F081E02DC6010995892B79F7C50171
:10013000DF91CF911F910F91FF90EF90DF90CF90C3
:10014000BF90AF900895FC0154894589252F30E078
:10015000842F90E0821B930B541710F0CF960895D4
:1001600001970895FC0192898389981761F0A3890A
:10017000AE0FBF2FB11D59968C9193899F5F9F73CE
:10018000938B90E008958FEF9FEF0895FC01928983
:100190008389981731F08389E80FF11D818D90E0F4
:1001A00008958FEF9FEF0895FC0192892389892F8D
:1001B00090E0805C9F4F821B91098F73992708956F
:1001C0008AE298E30E94D40021E0892B09F420E020
:1001D000822F089580E090E0892B29F00E94E000B2
:1001E00081110C9400000895CF93DF93EC01E88116
:1001F000F9810284F385E02D0995EC85FD858681E2
:100200008F738683EC85FD8585818F7585838B89CA
:100210008A8B198ADF91CF910895CF92DF92EF9266
:10022000FF920F931F93CF93DF93EC016A017B0141
:10023000022F8989882339F0E881F9810088F189C2
:10024000E02DCE0109951FB7F89460E078E689E8C3
:1002500099E0A70196010E943D042F5F3F4F4F4F49
:100260005F4F5695479537952795EC85FD85868197
:100270008D7F8683EC85FD8586818683198A8E85B0
:100280008C3020F590E0FC01E056FF4F64916F3F09
:10029000E9F0FC01EC56FF4FA49170E2A79FD0015A
:1002A0001124BC5FFC01E857FF4FE491EF3F09F4D4
:1002B00076C0CD014096E80FF92FF11D9FB7F89455
:1002C00012966C938081886080839FBF8F858C306D
:1002D00038F590E0FC01E056FF4FF4906FEFF61612
:1002E000F9F0FC01E458FF4F6491662351F0FC01E2
:1002F000E857FF4FE491613009F454C0693009F4C4
:1003000061C0FC01EC56FF4FA49170E2A79FD001A1
:100310001124BC5F6C916F2109F457C01596FC92B3
:100320008F858C3090F490E0FC01E056FF4F649193
:100330006F3F59F0FC01EC56FF4FA49180E2A89F5B
:10034000D0011124BC5F11966C93A09125110A2E47
:10035000000CBB0BBC5F0E945F04EC85FD852AE0AE
:1003600095958795779567952A95D1F760877187D9
:10037000EC85FD850783EC85FD858681806C868311
:10038000EC85FD858581806885831FBFDF91CF91D6
:100390001F910F91FF90EF90DF90CF900895F0E0C4
:1003A000E0E08CCFE33008F0EF5FF091010A61E00C
:1003B00070E001C0660FEA95EAF760956F236093DD
:1003C000010A9FCF1092A0069CCFFC01E857FF4F77
:1003D000E491109769F0EF3F59F05096EA0FFB2F28
:1003E000F11D9FB7F8948081886080839FBF98CF6C
:1003F000F0E0E0E0F6CFCF93DF93FC0194898589AC
:10040000C485D585981306C08D818F7D8D83DF913E
:10041000CF910895A589AE0FBF2FB11DA75ABF4F29
:100420002C91858990E001968F739927858B80E4C4
:100430008C83A485B58512962C93A485B5851496D6
:100440008C91149785FFFBCF948985899813DFCF12
:1004500015968C9115978F7D15968C938789882397
:10046000B1F2808D80931301178AD1CFEF92FF9262
:100470000F931F93CF93DF93EC0181E0898B9C89CD
:100480008D8998131CC0AC85BD8514968C911497EA
:1004900085FF15C012966C93AC85BD8580E41496DB
:1004A0008C93EC85FD8585818F7D858381E090E04F
:1004B000DF91CF911F910F91FF90EF900895809160
:1004C000110180FF08C080911301888F8E8980936D
:1004D000130181E08F8BF62E0C8910E00F5F1F4F08
:1004E0000F731127E02E8D898E110CC00FB607FEF9
:1004F00005C0EC85FD85858185FDF5CFCE010E9487
:10050000FB01F1CFEC89EC0FFD2FF11DE75AFF4FF6
:10051000F0820C8BEC85FD8585818062C6CFCF9300
:10052000DF93FC0121892223F9F0EC018091110174
:1005300080FF08C080911301808F8689809313010A
:1005400081E0878BEC85FD85858185FD03C08481F5
:1005500086FD0AC00FB607FE03C0858185FDF2CF78
:10056000CE010E94FB01EECFDF91CF91089581E093
:100570000895DC01ED91FC910684F785E02D23E0E0
:1005800030E00994FC0101900020E9F73197AF01B8
:10059000481B590BBC018AE298E30C9476001F9229
:1005A0000F920FB60F9211242F933F934F935F93A7
:1005B0006F938F939F93AF93BF93809126389091C1
:1005C0002738A0912838B09129384091243850918B
:1005D00025389A012D5C3C4F283E63E0360728F011
:1005E000285E33400196A11DB11D2093243830931D
:1005F00025388093263890932738A0932838B093D5
:1006000029388091203890912138A0912238B091DA
:1006100023380196A11DB11D809320389093213875
:10062000A0932238B093233881E080938D0ABF9144
:10063000AF919F918F916F915F914F913F912F91CA
:100640000F900FBE0F901F9018951F920F920FB62C
:100650000F9211242F933F934F935F936F937F9348
:100660008F939F93AF93BF93EF93FF938AE298E3A7
:100670000E94FB01FF91EF91BF91AF919F918F91EC
:100680007F916F915F914F913F912F910F900FBE8E
:100690000F901F9018951F920F920FB60F92112472
:1006A0002F938F939F93EF93FF93E0913638F091C0
:1006B0003738818181FD1BC0908180913C388F5FEC
:1006C0008F7320913D38821741F0E0913C38F0E083
:1006D000E65DF74C918F80933C38FF91EF919F91AD
:1006E0008F912F910F900FBE0F901F9018958081C2
:1006F000F4CF88ED90E084BF909361008091020672
:1007000086608093020680910006816080930006D7
:10071000809102068F7C809302068091A0008F78E2
:100720008093A0008091020680618093020621E000
:100730002093030A9EEF9093260A9093270A80E85D
:100740008093280A80932A0A80932C0A8093290A8E
:1007500080932B0A80932D0A3BE03093000A47E0F8
:100760004093410A90934C0A80934D0A35E03093B0
:10077000400A4093510A90935C0A80935D0A30933B
:10078000500A8FEF91E08093AE0A9093AF0A2093C6
:100790008C0A1092810A81E18093800A8091A000E6
:1007A0008093A000789440E052EC61E070E08AE22F
:1007B00098E30E94B902C0E0D0E08AE298E30E9488
:1007C000D4001816190674F58AE298E30E94B20064
:1007D00080931F388CE299E80E94C20280911D38F4
:1007E00090911E389C012F5F3F4F20931D3830930E
:1007F0001E388C5F974C40911F38FC014083283194
:10080000310521F410921D3810921E3884E098E3CF
:100810000E94C20288E499E80E94C2028AE499E830
:100820000E94C202209749F20E94E000882329F228
:100830000E940000C2CFEAE2F8E31282138288EE3F
:1008400093E0A0E0B0E084839583A683B78386E13C
:1008500099E88083918380E098E08487958784E09D
:10086000868785E08787108A128A138A148A158AF8
:100870008CE1868B178A108E0895A1E21A2EAA1B8E
:10088000BB1BFD010DC0AA1FBB1FEE1FFF1FA21740
:10089000B307E407F50720F0A21BB30BE40BF50B3D
:1008A000661F771F881F991F1A9469F760957095C6
:1008B000809590959B01AC01BD01CF010895B7FFD4
:1008C0000C946D040E946D04821B930B0895EE0F2F
:1008D000FF1F0590F491E02D09940E947804A59FD4
:1008E000900DB49F900DA49F800D911D112408952B
:1008F000A29FB001B39FC001A39F700D811D112461
:10090000911DB29F700D811D1124911D0895F894C1
:02091000FFCF17
:100912000000000036027600D400B200C6008F024A
:10092200B9020D01F400B702A30068656C6C6F2E6A
:1009320074313631342E6563686F3A20796F7520D1
:0B09420074797065642022000D0A002B
:00000001FF
